:1000000012C02CC02BC02AC029C028C027C026C0BF
:1000100025C024C023C022C021C020C01FC01EC0D4
:100020001DC01CC01BC011241FBECFE5D4E0DEBF25
:10003000CDBF10E0A0E6B0E0E8E0F2E002C005903D
:100040000D92A036B107D9F710E0A0E6B0E001C0EC
:100050001D92A037B107E1F760D0D5C0D1CFAC0178
:10006000892B59F020E030E08AEF90E00197F1F71A
:100070002F5F3F4F24173507B9F70895BB9ABC98F7
:10008000BD9A8A98BA9AA19A8B9A0895C29AC39AED
:10009000C59880B386B3A99A0895C598C29840E0E0
:1000A00020E030E0992314F4C39A01C0C398C59AA4
:1000B000220F331FB4992160C5984F5F403119F06A
:1000C000880F991FEFCFC598C29AC90108958299E8
:1000D000FECF90E080509844E0DF08958299FECFF3
:1000E000C598C298C39820E080E0880FB4998160D9
:1000F000C59AC5982F5F2831C1F7C29A90E008953C
:1001000010BC8CE089B988E18AB986E880BD599A2B
:1001100008955D9BFECF8CB908956F927F929F9258
:10012000AF92BF92CF92DF92EF92FF920F931F9305
:10013000CF93DF93A3DFE4DFA9DF84E690E08FDFD6
:1001400093988DE790E9A9DF80E496EAA6DF83E241
:1001500098ECA3DF8CEA94ECA0DF8BE696EC9DDFB5
:1001600080E090EC9ADF81E890EC97DF80E09EECF5
:1001700094DF99240F2EF0E6AF2EF0E0BF2EF02D85
:100180003501CC24DD246894C4F8CA0CDB1C8BE850
:100190009EEC83DF8501E301FF24A0DF8993F80E45
:1001A000CC15DD05D1F79ADFE82E98DF80E09EECD4
:1001B00074DFF80181918F01ACDF82E090E04FDFC6
:1001C000C017D107B1F7FE1441F4909480E2A1DF8B
:1001D0008FE69FDF8BE69DDF10C08AE09ADF82E02A
:1001E00090E03DDF8DE095DF82E090E038DF85E64E
:1001F00090DF82E78EDF82E78CDF992011F0939AFF
:08020000C6CF9398C4CFFFCFD5
:00000001FF
